:0400000000000000FC
:0400010000000000FB
:0400020000000000FA
:040003002EC6000005
:0400040017280A2788
:04000500190400AF2B
:0400060000000000F6
:0401000000000000FB
:040101002604202F81
:0401020000000000F9
:0402000000000000FA
:040201001EB286A8FB
:04020200328287A815
:0402030020C603E02E
:04020400188A06202E
:04020500030440812D
:0402060031C20740BA
:040207003EB2800083
:040208003EB2800082
:040209002D820740FB
:04020A002150000F70
:04020B002AC6000EF1
:04020C001B82E6AEBD
:04020D0038B226AF2E
:04020E003B20000091
:04020F002B0441EF8C
:0402100000000000EA
:0404000000000000F8
:0404010035C2078178
:04040200169016A991
:040403002150000F75
:0404040021C6004EBF
:040405001682E02E4D
:040406002150000F72
:040407002EC7FFE31A
:0404080004C6010F16
:0404090031B22021CB
:04040A001F8211EF4D
:04040B0008C600041B
:04040C0032C2078968
:04040D003EC207C123
:04040E002420120193
:04040F0019C2070106
:040410002DA41060A7
:040411002F0484D15F
:0404120007201200AD
:0404130000000000E5
:0404140009E6404174
:0404150039A6106193
:0404160000000000E2
:040417000FE640426A
:0404180010B280425C
:0404190010B280425B
:04041A0034AA2022BE
:04041B002820200075
:04041C00133C20006D
:04041D002B38200058
:04041E0013824624DB
:04041F00108847807A
:0404200037884120B8
:04042100260482909B
:040422000FE640425F
:040423002A048477AC
:0404240001282C1867
:040425000704868FB3
:040426001DB3F128E9
:0404270021B380215C
:0404280027B3802254
:040429003B7A0041D9
:04042A0032AA2021B1
:04042B000920100094
:04042C00323C10004E
:04042D000A38100079
:04042E0013824624CB
:04042F001D884100E3
:0404300024048641D9
:0404310003BE0021E5
:0404320037884120A6
:0404330007048570C5
:0404340037C207E0E4
:040435003B20000068
:04043600220486D73F
:04043700003C000085
:040438003838000050
:0404390022048737DB
:04043A00003C000082
:04043B00383800004D
:04043C002404879776
:04043D002EC60000C7
:04043E0017280A274A
:04043F002B0487EF14
:0404400000000000B8
:00000001ff
